:0200000480007A
:100000006F008004732F2034930F80006308FF0378
:10001000930F90006304FF03930FB0006300FF038E
:10002000130F000063040F0067000F00732F2034CC
:1000300063540F006F00400093E19153171F0000BD
:1000400023223FFC6FF09FFF732540F163100500F2
:10005000970200009382020173905230735000188F
:10006000970200009382020273905230B702008020
:100070009382F2FF7390023B9302F0017390023A75
:1000800097020000938282017390523073502030A7
:1000900073503030735040309301000097020000DD
:1000A000938282F673905230130510001315F501F8
:1000B000634C05000F00F00F930110009308D0056A
:1000C000130500007300000093020000638E02001D
:1000D00073905210B7B20000938292107390223046
:1000E00073232030E39A62F47350003097020000CB
:1000F0009382420173901234732540F173002030D3
:1001000093012000930000001301000063D620003B
:100110006318303063163000E3DE20FE63123030A7
:1001200093013000930010001301100063D62000EB
:100130006318302E63163000E3DE20FE6312302E8B
:10014000930140009300F0FF1301F0FF63D62000FD
:100150006318302C63163000E3DE20FE6312302C6F
:1001600093015000930010001301000063D620009B
:100170006318302A63163000E3DE20FE6312302A53
:1001800093016000930010001301F0FF63D620007C
:100190006318302863163000E3DE20FE6312302837
:1001A000930170009300F0FF1301E0FF63D620007D
:1001B0006318302663163000E3DE20FE631230261B
:1001C00093018000930000001301100063D420000D
:1001D0006314300063163024E3DE20FE93019000A8
:1001E0009300F0FF1301100063D42000631430006B
:1001F00063183022E3DE20FE9301A0009300E0FFAD
:100200001301F0FF63D4200063143000631A302020
:10021000E3DE20FE9301B0009300E0FF1301100025
:1002200063D4200063143000631C301EE3DE20FE24
:100230009301C000130200009300F0FF13010000BF
:1002400063D0201E1302120093022000E31652FE18
:100250009301D000130200009300F0FF130100008F
:100260001300000063DE201A130212009302200024
:10027000E31452FE9301E000130200009300F0FF2C
:1002800013010000130000001300000063DA2018BF
:100290001302120093022000E31252FE9301F000B9
:1002A000130200009300F0FF130000001301000090
:1002B00063D820161302120093022000E31452FEAA
:1002C00093010001130200009300F0FF13000000EF
:1002D000130100001300000063D420141302120065
:1002E00093022000E31252FE93011001130200005A
:1002F0009300F0FF13000000130000001301000042
:1003000063D020121302120093022000E31252FE67
:1003100093012001130200009300F0FF130100007D
:1003200063D020101302120093022000E31652FE45
:1003300093013001130200009300F0FF130100004D
:100340001300000063DE200C130212009302200051
:10035000E31452FE93014001130200009300F0FFEA
:1003600013010000130000001300000063DA200AEC
:100370001302120093022000E31252FE9301500177
:10038000130200009300F0FF1300000013010000AF
:1003900063D820081302120093022000E31452FED7
:1003A00093016001130200009300F0FF13000000AE
:1003B000130100001300000063D420061302120092
:1003C00093022000E31252FE930170011302000019
:1003D0009300F0FF13000000130000001301000061
:1003E00063D020041302120093022000E31252FE95
:1003F0009300100063DA00009380100093801000D7
:100400009380100093801000938010009380100060
:10041000930E3000930180016394D0016310300289
:100420000F00F00F638001009391110093E1110020
:100430009308D00513850100730000000F00F00F32
:10044000930110009308D00513050000730000000D
:10045000731000C000000000000000000000000059
:10046000000000000000000000000000000000008C
:0C04700000000000000000000000000080
:1010000000000000000000000000000000000000E0
:1010100000000000000000000000000000000000D0
:1010200000000000000000000000000000000000C0
:1010300000000000000000000000000000000000B0
:081040000000000000000000A8
:040000058000000077
:00000001FF
